:10000000E829FF3FFF3FFF3FC000030E8301A6002A
:100010004008A5000408A8000A08A7008A01C10139
:10002000051AC10A13084106C200C5010030C50601
:10003000C3014208430203194628940A0319950A8A
:10004000B030C0003630C1004108C2001708C202FB
:10005000031D2C2816084002031843289801C001EC
:100060001908400203193D281B089A001D089C002E
:100070009E019F01A0010130A1009B011B089D0072
:10008000A2019901A315960197017029960A0319F7
:10009000970AC001C1011508C102031D51281408A7
:1000A000400203186E297830C0000530C1004108B5
:1000B000C2001508C202031D5F281408400203187D
:1000C00009290130A40095289D0AE32802301D0764
:1000D0009D00E32804301D079D00E32808301D071C
:1000E0009D00E3280A301D079D00E32814301D07FA
:1000F0009D00E32828301D079D00E3289B0AE32884
:1001000002301B079B00E32804301B079B00E328F9
:1001100008301B079B00E3280A301B079B00E328DD
:1001200014301B079B00E328E3281530C00040086B
:100130001802031964281630C00040081802031979
:1001400066281730C0004008180203196A281830C2
:10015000C0004008180203196E281930C00040087A
:100160001802031972281A30C00040081802031937
:1001700076281B30C0004008180203197A281D3069
:10018000C0004008180203197E281E30C000400835
:100190001802031980281F30C000400818020319F4
:1001A00084282030C0004008180203198828213014
:1001B000C0004008180203198C282230C0004008F3
:1001C0001802031990281C30C000400818020130A2
:1001D00003190030C1004108031905292330C2006A
:1001E00042081802013003190030C5004508031900
:1001F00005293A30C30043081802013003190030C2
:10020000C40044080319052906290729A20A980AE7
:1002100029298030C0000230C1004108C200150801
:10022000C202031D152914084002031825291430A1
:10023000C00040081802031D2229FF30A4009801C5
:10024000A3112429A401980A2929FF30A4009801A8
:10025000A3111530C00040081802031D3029A20167
:100260001D30C000400818020130031D0030C100DD
:100270004108031D52292430C200420818020130EF
:10028000031D0030C5004508031D52293B30C30043
:10029000430818020130031D0030C4004408031D48
:1002A000522953295429672901302205C000C10170
:1002B0000030C1054108C2000030C202031D62299E
:1002C00024084002031966299801A311A2013B30BA
:1002D000C00040081802031D6E29990A9401950177
:1002E0009F0A0319A00A2630C0002630C10020084A
:1002F000C2004108C202031D7F2940081F02031DDE
:100300009E296030010781009F01A0019E0A3C30B8
:10031000C00040081E02031D9E299E019C0A3C301D
:10032000C00040081C02031D9E299C019A0A183037
:10033000C00040081A02031D9E299A01C001051A37
:10034000C00A13084006C100A3104118A3140B11E2
:100350002508C00027088A0028088400260E83008C
:10036000C00E400E0900080003138312A3013F30A2
:10037000AE000630AF005B30B0004F30B1006630E9
:10038000B2006D30B3007C30B4000730B5007F3070
:10039000B6006730B70038309E0022309C000C3029
:1003A0009A0001309300A1019901980108000313FC
:1003B00083128C0108309200100D8C0D0E088C02F7
:1003C0000318E4298C070310900D920BDC29080018
:1003D000B42110300313831685008601A0308B00F2
:1003E000D830810003138312C70121084702031884
:1003F000C12AC701290847020319592A2A30C70010
:100400000A308E001C089000D7211008C8002E303A
:10041000C9004808C907490884000008CA004708FD
:1004200084004A0880002A30C7000130C7070A301C
:100430008E001C089000D7210C08C8002E30C9007F
:100440004808C907490884000008CA004708840012
:100450004A0880002A30C7000230C7070A308E00E1
:100460001E089000D7211008C8002E30C900480887
:10047000C907490884000008CA00470884004A08E0
:1004800080002A30C7000330C7070A308E001E08DC
:100490009000D7210C08C8002E30C9004808C907B1
:1004A000490884000008CA00470884004A08800000
:1004B000C02A2A30C7000A30C80048081A02013092
:1004C00003180030CB004B080319682AC901772AAA
:1004D0000A308E001A089000D7211008CA002E306A
:1004E000CC004A08CC074C0884000008C900470823
:1004F0008400490880002A30C7000130C7070A304D
:100500008E001A089000D7210C08C8002E30C900B0
:100510004808C907490884000008CA004708840041
:100520004A0880002A30C7000230C7070A308E0010
:100530001C089000D7211008C8002E30C9004808B8
:10054000C907490884000008CA00470884004A080F
:1005500080002A30C7000330C7070A308E001C080D
:100560009000D7210C08C8002E30C9004808C907E0
:10057000490884000008CA00470884004A0880002F
:10058000FA2A2A30C700840080012A30C7000130CF
:10059000C7074708840080012A30C7000230C70718
:1005A0000A308E0018089000D7211008C8002E309D
:1005B000C9004808C907490884000008CA0047085C
:1005C00084004A0880002A30C7000330C7070A3079
:1005D0008E0018089000D7210C08C8002E30C900E2
:1005E0004808C907490884000008CA004708840071
:1005F0004A0880002A30C7002308C8000130C80517
:10060000470884008013481880172A30C70001303B
:10061000C707C801A318C80A4708840080134818F0
:1006200080172A30C7000230C707C8012319C80A3B
:10063000470884008013481880172A30C700033009
:10064000C707C801A319C80A4708840080134818BF
:10065000801785018601803083168600C7018312CA
:10066000861BC70A4708A90083168601B80A03300B
:10067000C700380847020318412BB8010130B90000
:10068000532B0130C7004708C8000030C81BFF309B
:10069000CB0038080319512BC80DCB0D4810FF3F74
:1006A0004A2B4808B9002A30C7003808C70747084E
:1006B000840000088312860039088500F2295F2B28
:10420000FF00FF00FF00FF00FF00FF00FF00FF00B6
:10421000FF00FF00FF00FF00FF00FF00FF00FF00A6
:10422000FF00FF00FF00FF00FF00FF00FF00FF0096
:10423000FF00FF00FF00FF00FF00FF00FF00FF0086
:10424000FF00FF00FF00FF00FF00FF00FF00FF0076
:10425000FF00FF00FF00FF00FF00FF00FF00FF0066
:10426000FF00FF00FF00FF00FF00FF00FF00FF0056
:10427000FF00FF00FF00FF00FF00FF00FF00FF0046
:10428000FF00FF00FF00FF00FF00FF00FF00FF0036
:10429000FF00FF00FF00FF00FF00FF00FF00FF0026
:1042A000FF00FF00FF00FF00FF00FF00FF00FF0016
:1042B000FF00FF00FF00FF00FF00FF00FF00FF0006
:1042C000FF00FF00FF00FF00FF00FF00FF00FF00F6
:1042D000FF00FF00FF00FF00FF00FF00FF00FF00E6
:1042E000FF00FF00FF00FF00FF00FF00FF00FF00D6
:1042F000FF00FF00FF00FF00FF00FF00FF00FF00C6
:02400E00FA3F77
:00000001FF
